:1000000012C0189518951895189518951895189563
:100010001895189518951895189518951895189578
:100020001895189518958FE58DBFC0E4E8E34E2E1E
:1000300084E08EBFD4E0F4E05F2EEEEFF3E0A0E6C4
:10004000B0E0A89584B7082E877F84BF88E1992700
:1000500081BD91BD88278D933197E9F76624B99AC0
:10006000BA9A83EA8FBD81E08EBD8FEF87BB8FEF99
:1000700084BB80E081BBA99AAA98AB9AAC988FEF19
:1000800093E090934B0080934A008FEF93E090931E
:10009000490080934800EFCFF894FFCF3197F1F7F4
:0E00A0000895689462F80895E89462F808954F
:00000001FF
